:020000020000FC
:10000000F5C0014285C040627894339402C098BB29
:10001000189547FD88BB09F541FD09C040FD1DC08D
:100020006A9591F400E008BB00E705BF189543FF0F
:1000300002C0446001C0C1D040FD0FC06A9521F4E8
:100040004D7F87E097E06AE040582AF002E009BF60
:1000500000E008BB02C00AE009BF40FD1AD0F894D6
:100060004F7D44FF1895AED04F7E1895152F110F78
:10007000110F19BD99E0552351F08AE0503440F03A
:100080009AE031F08CE0503818F09CE009F089E0FB
:1000900008956A9551F44E77877F977F02E009BFF4
:1000A00000E008BB6EE041FF6AE0089522241127BA
:1000B0009D01369527951795369527951795211A01
:1000C000A20BB30B18E0220CAA1FBB1F18F0A81537
:1000D000B90518F0A819B90923941A95A1F708953C
:1000E000AA19BB0918F0AC19BD09E8F7AC0DBD1D84
:1000F000460114E0969487941A95E1F7811E911EAB
:10010000A819B909E8F7A80DB91DD0DF522DAECF57
:10011000A2B7B32D18B711FDAFEF10E215BFCA1B80
:10012000DB0BCA361FEFD10728F4ED01B49B03C0E7
:1001300048604D0118954FB6477FA815B9051FB700
:10014000A80DB91DB795A79510FDB058A019B10914
:100150000A0E1B1EA5301DE0B10748F5A33019E0BB
:10016000B10728F140FD0AC0416841FD03C02224C7
:10017000DD24CC24886098600AE009BF41FD13C0EB
:10018000222059F02A1B3B0B285D3F4F2055304061
:1001900020F02224DD24CC240AC09D01CA0EDB1EDF
:1001A000239425FE04C045FF0DD045FD406140FD70
:1001B00067E142FD02D04FBE1895AC0CBD1CE8F7BC
:1001C0004B7F0895D00141FF05C0B7FD89CF42FDA7
:1001D000F4DF86CF42600894D794C794AC19BD0968
:1001E000E8F7AC0DBD1D5D01552740CF0FE90DBFF0
:1001F000479A03E00FBD02E003BF0FE007BB00E139
:1002000005BB0AE009BF00E205BF0BBF40E86AE09A
:0A02100087E097E078948895FECF10
:00000001FF
